:100000000C9434000C9451000C9451000C94510049
:100010000C9451000C9451000C9451000C9451001C
:100020000C9451000C9451000C9451000C9451000C
:100030000C9451000C9451000C9451000C945100FC
:100040000C9451000C9451000C9451000C945100EC
:100050000C9451000C9451000C9451000C945100DC
:100060000C9451000C94510011241FBECFEFD4E02A
:10007000DEBFCDBF12E0A0E0B1E0EAE6F9E002C0E9
:1000800005900D92AE3FB107D9F712E0AEEFB2E0A6
:1000900001C01D92AE3FB107E1F70E9423040C940A
:1000A000B3040C94000020E030E087FF02C0599AAE
:1000B00001C059985C985C9A2F5F3F4F28303105FA
:1000C00011F0880FF2CF59980895299841980E940D
:1000D0005300419A0895429880E090E02AEF30E082
:1000E000F9013197F1F701968A309105C9F7429AE3
:1000F00080E090E02AEF30E0F9013197F1F70196C6
:10010000883C9105C9F785E10E94650087E00E945F
:10011000650089E30E94650085E70E94650080E034
:100120000E9465008FE40E94650086E80E946500D9
:1001300081E80E9465008DE20E9465008EEB0E94BE
:10014000650081E10E9465008CEB0E9465008FE0F4
:100150000E94650080EA0E94650081E40E946500BB
:1001600086EA0E94650088EA0E9465008FE40E948A
:10017000650081EB0E94650082E20E94650082EBCF
:100180000E94650086E40E94650080EB0E94650085
:1001900088E00E94650084EB0E94650080E00E9478
:1001A000650083EB0E94650080EA0E9465008FEB8A
:1001B0000E9465008DE00E94650088EB0E9465004A
:1001C00081E00E94650081E10E94650082E20E9458
:1001D000650082E30E94650083E40E94650084E577
:1001E0000E94650085E60E94650086E70E94650022
:1001F0008EEA0E9465008DEA0E94650082E00E94FE
:10020000650080E090E02AEF30E0F9013197F1F7E6
:1002100001968B349105C9F784EA0E9465008FEA44
:100220000E94650083EE0E94650008952998419A16
:100230000E945300299A08954F925F926F927F9285
:100240008F929F92AF92BF92CF92DF92EF92FF92E6
:100250000F931F93CF93DF93C82E662ED42E85E184
:100260000E946500E8E08E2E860C882D0E946500B5
:1002700070E1772E760C872D0E94650085E70E943D
:1002800065008D2D0E9465008D2D8C5F0E9465009C
:10029000FF2421E0C21611F4FF24F39480E044E02F
:1002A000C41609F481E09F2C982A19F4C0EDD2E01D
:1002B00021C010E080E00E9416011F5F1432D1F7C8
:1002C0001DC0202F2695822F8E2111F490E001C0B1
:1002D00090EF022F0695802F8E2109F09F60892FC5
:1002E0000E9416011F5F143061F7219682E0C93D1C
:1002F000D80721F0E88020E810E0E5CF85E10E94F2
:100300006500882D0E946500872D0E94650085E7A5
:100310000E9465008D2D8E5E0E9465008D2D8B5E86
:100320000E946500EE2497E0C91611F4EE24E394D0
:10033000AA24BB24CC2019F461E0A62EB12CFE28FF
:100340008F2D90E08A299B29892B19F4C9EDD2E0E1
:1003500021C010E080E00E9416011F5F1432D1F727
:100360001DC0202F2695822F8F2111F490E001C00F
:1003700090EF022F0695802F8F2109F09F60892F23
:100380000E9416011F5F143061F7219622E0C23EE1
:10039000D20721F0F88020E810E0E5CF85E10E9447
:1003A0006500882D0E946500872D0E94650085E705
:1003B0000E9465008D2D8C5D0E9465008D2D895DEC
:1003C0000E946500892D90E020E030E047E0C416EF
:1003D00011F421E030E0822B932B892B19F4C2EE2B
:1003E000D2E021C010E080E00E9416011F5F1432AD
:1003F000D1F71DC0202F2695822F8F2111F490E078
:1004000001C090EF022F0695802F8F2109F09F6089
:10041000892F0E9416011F5F143061F7219682E038
:10042000CB3ED80721F0F88010E020E8E5CF85E149
:100430000E94650057E0952E960C892D0E9465005C
:10044000882D0E94650085E70E94650042E0442EE9
:100450004D0C842D0E94650033E1532E5D0C852DDB
:100460000E9465008C2D8150833028F0EE2019F415
:10047000CBEED2E021C010E080E00E9416011F5FA9
:100480001432D1F71DC0202F2695822F8F2111F411
:1004900090E001C090EF022F0695802F8F2109F088
:1004A0009F60892F0E9416011F5F143061F721960B
:1004B00092E0C43FD90721F0F88010E020E8E5CFB2
:1004C00085E10E946500892D0E946500882D0E94AB
:1004D000650085E70E94650024E1822E8D0C882D41
:1004E0000E94650095E2992E9D0C892D0E94650061
:1004F000EE2422E0C21611F4EE24E39480E090E0B2
:1005000048E0C41611F481E090E09C012A293B29BF
:1005100080E096E0C91609F481E08E2990E0282B4E
:10052000392B232B01F1CBEED2E019C0202F2695D9
:10053000822F8F2111F490E001C090EF022F0695D9
:10054000802F8F2109F09F60892F0E9416011F5F65
:10055000143061F7219622E0C43FD20759F0F880A9
:1005600010E020E8E5CF10E080E00E9416011F5F58
:100570001432D1F785E10E946500872D0E94650045
:1005800081E1D82ED60C8D2D0E94650085E70E9452
:100590006500842D0E946500852D0E9465004BEF4B
:1005A000C40E81E08C1518F4C4EFD2E021C010E035
:1005B00080E00E9416011F5F1432D1F71DC0202F6A
:1005C0002695822F8F2111F490E001C090EF022F29
:1005D0000695802F8F2109F09F60892F0E941601B8
:1005E0001F5F143061F7219692E0CD3FD90721F0CB
:1005F000F88010E020E8E5CF85E10E946500872DB6
:100600000E9465008D2D0E94650085E70E946500AF
:10061000882D0E946500892D0E946500EE2019F446
:10062000C4EFD2E021C010E080E00E9416011F5FFD
:100630001432D1F71DC0202F2695822F8F2111F45F
:1006400090E001C090EF022F0695802F8F2109F0D6
:100650009F60892F0E9416011F5F143061F7219659
:1006600022E0CD3FD20721F0F88010E020E8E5CF6E
:10067000DF91CF911F910F91FF90EF90DF90CF907E
:10068000BF90AF909F908F907F906F905F904F90B2
:1006900008956F927F928F929F92AF92BF92CF9266
:1006A000DF92EF92FF920F931F93982F062FF42E55
:1006B0008052803608F090E2E5E09E9FF001112420
:1006C000E05AF040DF01A75FBE4F6C903196DF012A
:1006D000A75FBE4F7C903196DF01A75FBE4F8C9025
:1006E000E65FFE4F9080A18085E10E94650016E0E4
:1006F000019F102D1124812F875F0E946500812F9B
:10070000835F0E94650085E70E9465008F2D90E061
:10071000F4E0880F991FFA95E1F7182F0E94650001
:10072000812F815F0E94650011E0BB24812F86210B
:1007300011F4CC2402C0CC24CA94812F872111F457
:10074000DD2402C0DD24DA94812F882111F4EE2407
:1007500002C0EE24EA94812F892111F4FF2402C003
:10076000FF24FA94812F8A2111F400E001C00FEFD9
:100770008C2D0E9416018D2D0E9416018E2D0E9437
:1007800016018F2D0E941601802F0E9416018C2DBC
:100790000E9416018D2D0E9416018E2D0E941601B9
:1007A0008F2D0E941601802F0E941601B39488E0BD
:1007B000B81611F0110FBACF1F910F91FF90EF9063
:1007C000DF90CF90BF90AF909F908F907F906F9071
:1007D0000895CF93DF9385E10E94650087E00E9432
:1007E000650089E30E94650085E70E94650080E05E
:1007F0000E9465008FE40E946500C0E0D0E080E0C8
:100800000E94160121968FE0C03FD807C1F7DF9103
:10081000CF9108950F931F93CF93DF93062FEA0193
:10082000682F07C0162F1F5F402F0E944903219693
:10083000612F8881882311F06131A0F3DF91CF917E
:100840001F910F910895EF92FF920F931F93CF93F3
:10085000DF93219A3A9A399A549A519A559A5D9A05
:1008600080E090E02AEF30E0F9013197F1F701964E
:1008700043E0883E9407C1F70E946B0080E090E05F
:100880002AEF30E0F9013197F1F7019684369105AE
:10089000C9F70E94E90380E060E040E051E00E9477
:1008A0000A0488E060E04EE10E941C0188E06DE0EF
:1008B0004EE10E941C0188E06AE14EE10E941C01A9
:1008C00088E067E24EE10E941C0180E090E02AEFA0
:1008D00030E0F9013197F1F7019643E0883E940743
:1008E000C1F7EE24CAEFD0E08E2D60E04EE10E9409
:1008F0001C01FF248F2D6DE04EE10E941C0100E0E1
:10090000802F6AE14EE10E941C0110E0812F67E216
:100910004EE10E941C0180E090E0FE013197F1F76A
:10092000019623E0883E9207C1F71F5F1A3071F7E6
:100930000F5F0A3029F7F3944AE0F416D9F6E394EE
:1009400089E08E1588F6EE24CFCF20E030E04AEF24
:1009500050E005C0FA013197F1F72F5F3F4F28179C
:0A0960003907C0F30895F894FFCFA3
:10096A005A6165686C65723A000000000000000078
:10097A002F00000007000700147F147F14242A7F29
:10098A002A12C4C8102646364955225002050200CA
:10099A0000001C2241000041221C0014083E0814D9
:1009AA0008083E080800005030001010101010000F
:1009BA006060000020100804023E5149453E004292
:1009CA007F40004261514946224149493618141272
:1009DA007F1027454545393C4A4949300171090587
:1009EA00033649494936064949291E003636000068
:1009FA00005636000008142241001414141414007E
:100A0A00412214080201510906324959513E7E1108
:100A1A0011117E7F494949363E414141227F414178
:100A2A00221C7F494949417F090909013E41494937
:100A3A007A7F0808087F00417F41002040413F013A
:100A4A007F081422417F404040407F020C027F7F92
:100A5A000408107F3E4141413E7F090909063E4193
:100A6A0051215E7F09192946464949493101017FC9
:100A7A0001013F4040403F1F2040201F3F40384077
:100A8A003F63140814630708700807615149454316
:100A9A00007F414100552A552A550041417F0004F3
:100AAA000201020440404040400001020400205478
:100ABA005454787F484444383844444420384444A1
:100ACA00487F3854545418087E0901020C52525275
:100ADA003E7F0804047800447D40002040443D00E5
:100AEA007F1028440000417F40007C041804787C71
:100AFA000804047838444444387C1414140808144C
:100B0A0014187C7C080404084854545420043F44B4
:100B1A0040203C4040207C1C2040201C3C4030406F
:100B2A003C44281028440C5050503C4464544C44D3
:100B3A003FFF1FFFE3FFF07FF81FFE0FFFC3FFF029
:100B4A007FF81FFE0FFFC7FFF8FFFC04EFFFFFFF50
:0E0B5A00FFFFFE40027FFFFFFFFFFFF72000BE
:00000001FF
